:10000000BB29A700B5008316061083120930B6007D
:1000100003101120B50CB60B092803141120270872
:10002000C728031816280000061044280614442880
:100030008830B1001330B200B501831686158312E3
:100040000000861D3228FF30B507031CB107031CD2
:10005000B207031CC728350A7D300319B50000001C
:1000600031282028B2010B3066200830B600442029
:10007000031086190314B50C00003E28B60B372870
:10008000442003143508C7282F3065289818181203
:1000900018168C1E49281A080314C728211B01288A
:1000A000080083169B0083161C141A089B0AC72895
:1000B000B601B500FF30B507031CB607031CC728FF
:1000C0000330B200E53066205A28B201F63EB10096
:1000D000B209031C7128FE300000B10703186C2818
:1000E000B1070000B20F6B280000311877283118D3
:1000F00079280800013EBA000A30B500B601842014
:10010000BA0B7F2837080800B801B7011030B900D2
:10011000320DB70DB80D3508B7023608031C360F7F
:10012000B80203189A283508B70736080318360F9F
:10013000B8070310B10DB20DB90B88283108C728D4
:100140001030BC00B201B101BA0CB90C031CAE28CE
:100150003508B10736080318360FB207B20CB10CD8
:10016000B80CB70CBC0BA4283708C728B100B41BC7
:10017000BB203108C728B109B209B309B409B10AD3
:100180000319B20A0319B30A0319B40A0800831346
:1001900083120313000008002908031D2D0803190A
:1001A000B5292A082E06C5002D08A9077E30031C94
:1001B000DD28A9020318AA29E028A902031C9F2907
:1001C0002A08C1002B08BF002C08C000C117AE17B9
:1001D0000310AA01AB01AC011830C400401CFA287E
:1001E0003008AC072F0803182F0FAB072E08031891
:1001F0002E0FAA07AA0CAB0CAC0CC10CBF0CC00C88
:100200000310C40BEE28AA1B0A29C10DAC0DAB0DBF
:10021000AA0DA903431B2C1C1C29C11F1C29AC0AB5
:100220000319AB0A0319AA0A031D1C29AA0CAB0C5B
:10023000AC0CA90A0319AA29C51FAA13003429085E
:10024000C100A9014108031900342A08C500AA17F2
:100250009E30C102C11F8529C109C10A083041026F
:10026000031C5A29C100A90D2C08A9002B08AC00B9
:100270002A08AB00AA0108304102031C5A29C10018
:10028000A90D2C08A9002B08AC00AB0108304102D5
:10029000031C5A29C100A90D2C08A900AC01083083
:1002A0004102031C5A29C100A90DA9014108031DDF
:1002B000031064294108031964290310AA0CAB0C2C
:1002C000AC0CA90CC10B5D29431B291C7229031C12
:1002D0007229A90A0319AC0A0319AB0A0319AA0A5D
:1002E000AA1B9229C51F9D29AA09AB09AC09A90916
:1002F000A90A0319AC0A0319AB0A0319AA0A9D2912
:10030000AA01AB01AC01A9019D294314C31F9D297A
:10031000AA01C51FFF30AA00AB00AC00A900C50DA3
:10032000AA0C9D294314C31FFF34AA01C51FFF3027
:10033000AA00AB00AC00C50DAA0C290808004315A3
:10034000C31FFF340130A900AA01AB01AC01C50DE8
:10035000AA0CFF34C314C31FFF34FF30A900AA0046
:10036000AB00AC00C50DAA0CFF34AA01AB01AC0177
:10037000C101A901003483160F3099002030980084
:100380008312803098006030C300A00107309F00C6
:10039000A030831685000A30860083128A156828EB
:1003A000F2018A0118208A11031CE229F2000630AA
:1003B00072028A11031DE0290130F8008A11E12937
:1003C000F80108000230F800080045308A010120D9
:1003D000080073088A015120F30042308A0101208D
:1003E00073088A010120080046308A01012002308A
:1003F0008A010120080074308A01012079088A01ED
:1004000001207E088A0101207F088A0101208316CD
:10041000200883128A0101208316210883128A0191
:10042000012074088A01012077088A0101207708D9
:100430008A0101208A01D021013078028A11031932
:10044000232A8A01FB290800BA017708B900B601FE
:100450000530B5008A01A020BD003808BE00143068
:100460003D078316C6008312BA0183163108831232
:10047000B900B601831646088312B5008A01A02090
:10048000BD003808BE0014303D078316A600831255
:100490003E080318013E8316A70027088312FE00BA
:1004A000831627088312B200831626088312B10030
:1004B0000130B600B5018A0184203708FF00831699
:1004C0002908A00029088312B20083162808831285
:1004D000B1000130B600B5018A01842037088316C7
:1004E000A100831208008316E0088A118312031DFD
:1004F0007F2A3F308316E10083128A11822A383026
:100500008316E1008312831627088312FE008316E8
:1005100027088312B200831626088312B100013027
:10052000B600B5018A0184203708FF008316290828
:10053000A00029088312B200831628088312B10094
:100540000130B600B5018A01842037088316A10066
:100550002B08A2002B088312B20083162A088312EC
:10056000B1000130B600B5018A0184203708831636
:10057000A3002D08A4002D088312B20083162C08B6
:100580008312B1000130B600B5018A01842037081A
:100590008316A500831262308A0101208316600849
:1005A00083128A0101207E088A0101207F088A01C6
:1005B00001208316200883128A0101208316210856
:1005C00083128A0101208316220883128A010120E6
:1005D0008316230883128A010120831624088312BC
:1005E0008A0101208316250883128A0101208316BF
:1005F000610883128A0101208A01D021013078022A
:100600008A110319052B8A01CA2A17308316A607F7
:100610000318A70A0A30A8070318A90A2708831293
:10062000FE00831627088312B20083162608831261
:10063000B1000130B600B5018A0184203708FF00FF
:1006400083162908A00029088312B20083162808FF
:100650008312B1000130B600B5018A018420370849
:100660008316A100831274308A01012079088A015F
:1006700001207E088A0101207F088A01012083165B
:10068000200883128A0101208316210883128A011F
:10069000012074088A01012001308A010120013003
:1006A0008A0101208A01D021013078028A110319C0
:1006B0005B2B8A01322B0800BA017708B900B6011A
:1006C0000E30B5008A01A020BD003808BE007C08AD
:1006D0003D078316A80083127D080318013E3E07DC
:1006E0008316A90083128A0124228A01FB210800B3
:1006F000BA017708B900B6011C30B5008A01A02004
:10070000BD003808BE007C083D078316A800831290
:100710007D080318013E3E078316A90083128A0153
:1007200024228A01FB210800BA017708B900B6012A
:100730002E30B5008A01A020BD003808BE007C081C
:100740003D078316A80083127D080318013E3E076B
:100750008316A90083128A0124228A01FB21080042
:10076000BA017708B900B6013C30B5008A01A02073
:10077000BD003808BE007C083D078316A800831220
:100780007D080318013E3E078316A90083128A01E3
:1007900024228A01FB2108005330831632028A1179
:1007A0008312031DD72B7608F4008A11D92B750804
:1007B000F400F9018316AE01B10183127D0883169E
:1007C000A90083127C088316A80083127B08831675
:1007D000A70083127A088316A60001305D028A11F1
:1007E0008312031DF62B12308316C3008312831667
:1007F00043082E0783128A015120F900F9088A1153
:100800000319062C8A0194238316B10A83128316D6
:10081000AE0A8312F9088A11031DF72B0800F901AB
:100820008316AE01B10183127D088316A9008312DD
:100830007C088316A80083127B088316A700831206
:100840007A088316A6008312173083162E078312A8
:100850008A015120F900F9088A110319332C8A0101
:100860005C238316B10A83128316AE0A8312F90839
:100870008A11031D232C0800F9018316AE01B10172
:1008800083127D088316A90083127C088316A800B2
:1008900083127B088316A70083127A088316A600AA
:1008A000C50101305D028A118312031D702C83166D
:1008B000C70183121F308316470783128A01512014
:1008C000A80083164708463E84008312280880004B
:1008D0008316C70A0B3047028A118312031D592C55
:1008E00083162E08463E840000088312F90031303A
:1008F00079028A11031C7F2C01308316DB008312DE
:100900003A3079028A11031D872C8316DB0183128A
:1009100083162E085C3E84000008C8008312790804
:10092000831648028A1183120319AC2C83162E08F1
:100930005C3E84008312790880008316DB088A11EC
:100940008312031DAA2C303079028A11031DAA2CB0
:100950002030F9008A01B0238316B10AAE0AC50A15
:100960000B302E028A118312031D702C0800F9012E
:100970008316AE01B10183127D088316A90083128C
:100980007C088316A80083127B088316A7008312B5
:100990007A088316A600C501831283162E08513EDD
:1009A000840000088312F900313079028A11031C97
:1009B000DC2C01308316DB0083123A3079028A1175
:1009C000031DE42C8316DB01831283162E08673E79
:1009D00084000008C80083127908831648028A112F
:1009E00083120319092D83162E08673E8400831293
:1009F000790880008316DB088A118312031D072DF6
:100A0000303079028A11031D072D2030F9008A0148
:100A100078238316B10AAE0AC50A0B302E028A115A
:100A20008312031DCC2C080083165C085F06023974
:100A30008A1183120319412D8A1183168310DC1C3D
:100A4000831483128318292D8316E00183128A11DF
:100A50002C2D01308316E00083125230F900023051
:100A60008316A7000F30A600A9013A30A800023073
:100A7000AB004430AA00AD015B30AC0083128A01A8
:100A8000732283165C085F0604398A1183120319E6
:100A90006E2D8A11831683105C1D831483128318B4
:100AA000562D8316E00183128A11592D01308316C9
:100AB000E00083124C30F90001308316A700A43007
:100AC000A600A9013A30A8000130AB00D930AA0035
:100AD000AD015B30AC0083128A01732283165C087F
:100AE0005F0608398A11831203199B2D8A11831618
:100AF0008310DC1D831483128318832D8316E00179
:100B000083128A11862D01308316E000831255303E
:100B1000F90001308316A700D930A600A9010A30D8
:100B2000A8000230AB000F30AA00AD012B30AC00A2
:100B300083128A01732283165C085F0610398A11BA
:100B400083120319C82D8A11831683105C1E831427
:100B500083128318B02D8316E00183128A11B32DFE
:100B600001308316E00083124430F900013083160F
:100B7000A700D930A600A9016A30A8000230AB0056
:100B80000F30AA00AD018B30AC0083128A017322B2
:100B900083165C08DF0083120800AC01AB01203033
:100BA000AA008230A900831636088312B00083168B
:100BB00035088312AF00831634088312AE00831603
:100BC00033088312AD008A01CC208A011F212C0832
:100BD0008316CA00831229088316C9008312AC0148
:100BE000AB012030AA008230A90083163A08831294
:100BF000B000831639088312AF00831638088312B9
:100C0000AE00831637088312AD008A01CC208A011A
:100C10001F212A088316D80083122B088316D700B9
:100C200083122C088316D600831229088316D50058
:100C30008A118310D81F831483128318252E013044
:100C40008316D90083128A11272E8316D9018312A5
:100C5000831658088312B400831657088312B30012
:100C6000831656088312B2008316550883128A0130
:100C7000B6208316CB00831232088316CC00831271
:100C8000AC01AB012030AA008230A90083163E08D7
:100C90008312B00083163D088312AF0083163C0810
:100CA0008312AE0083163B088312AD008A01CC206C
:100CB0008A011F212C088316CE008312290883166F
:100CC000CD008312AC01AB012030AA008230A90014
:100CD000831642088312B000831641088312AF00C6
:100CE000831640088312AE0083163F088312AD00BE
:100CF0008A01CC208A011F212A088316D40083127E
:100D00002B088316D30083122C088316D20083127B
:100D100029088316D1008A118310D41F83148312EB
:100D20008318982E01308316DA0083128A119A2EC6
:100D30008316DA018312831654088312B4008316D3
:100D400053088312B300831652088312B20083162D
:100D5000510883128A01B6208316CF00831232080D
:100D60008316D000C6010330C700831205308316F6
:100D700046028A1183120318F22E83164A08831240
:100D8000B200831649088312B10083164708831204
:100D90008A017A208316C8003030C80730304802F4
:100DA0008A1183120318D72E20308316C8008312AD
:100DB00083164608463E840048088000C60A033071
:100DC00046028A118312031DEC2E83164608463E06
:100DD00084002E308000C60A83128316C703831254
:100DE0008A01B52E03308316C7004608463E8400AC
:100DF0003A308000C60A013059028A118312031D5D
:100E0000092F83164608463E84002D308000C60A0E
:100E1000C70383120B30831646028A11831203180C
:100E2000462F83164C088312B20083164B08831298
:100E3000B1008316470883128A017A208316C800FE
:100E40003030C807303048028A11831203182B2F24
:100E500020308316C800831283164608463E84005D
:100E600048088000C60A093046028A118312031D11
:100E7000402F83164608463E84002E308000C60A66
:100E800083128316C70383128A010A2F8316C601B1
:100E90000330C70083120530831646028A1183127D
:100EA0000318872F83164E088312B20083164D084D
:100EB0008312B1008316470883128A017A208316B1
:100EC000C8003030C807303048028A118312031836
:100ED0006C2F20308316C800831283164608513EBB
:100EE000840048088000C60A033046028A11831233
:100EF000031D812F83164608513E84002E3080004A
:100F0000C60A83128316C70383128A014A2F03304D
:100F10008316C7004608513E84003A308000C60A56
:100F200001305A028A118312031D9E2F8316460830
:100F3000513E84002D308000C60AC70383120B3057
:100F4000831646028A1183120318DB2F831650087A
:100F50008312B20083164F088312B100831647082C
:100F600083128A017A208316C8003030C8073030D7
:100F700048028A1183120318C02F20308316C8003C
:100F8000831283164608513E840048088000C60A32
:100F9000093046028A118312031DD52F8316460895
:100FA000513E84002E308000C60A83128316C70388
:100FB00083128A019F2F08008A014620563C8A111D
:100FC000031DDC2F8A014620473C8A11031DDC2FBC
:100FD0008A014620413C8A11031DDC2F8A014620EC
:100FE0008316B20083128A0146208316B30083124F
:100FF0008A0146208316B40083128A014620831694
:10100000B50083128A0146208316B60083128A0136
:1010100046208316B70083128A0146208316B80043
:1010200083128A0146208316B90083128A01462062
:101030008316BA0083128A0146208316BB008312EE
:101040008A0146208316BC0083128A01462083163B
:10105000BD0083128A0146208316BE0083128A01D6
:1010600046208316BF0083128A0146208316C000E3
:1010700083128A0146208316C10083128A0146200A
:101080008316C2001E303205DC008A158310321F21
:10109000831483128318522801308316DD008312D3
:1010A0008A1554288316DD0183128A15831683104E
:1010B000B21F83148312831863284D308316B20045
:1010C00083128A15662853308316B20083120800F3
:1010D0000530B600DC308A0159208316C401FF3088
:1010E000DF00003083128A0151208316C60083126C
:1010F000BA01831646088312B900B6010A30B5005A
:101100008A01A0208316AF00831238088316B0002E
:10111000063083128A0151208316C6008312BA0159
:10112000831646088312B900B6010A30B5008A0159
:10113000A020FA003808FB0007308A0151208316EE
:10114000C6008312BA01831646088312B900B6019D
:101150000A30B5008A01A020FC003808FD000130EB
:101160008A015120F30003308A015120F500043038
:101170008A015120F60005308A015120F7005530D0
:101180008A0101208A01D021013078028A150319D1
:10119000CB288A15BF2842308A01012073088A01B2
:1011A00001208A01D021013078028A150319DA283A
:1011B0008A15CB288A01E5218A01D02101307802E5
:1011C0008A150319E5288A15DA284F308A0101208B
:1011D00001308A0101208A01D021013078028A156C
:1011E0000319F4288A15E5288A01DC278A01CD2510
:1011F0004D30831632028A158312031D07290830E9
:101200008316C3008312061686128A150D290D3027
:101210008316C3008312861606127D088316A90062
:1012200083127C088316A80083127B088316A7000C
:1012300083127A088316A600440832028A158312A4
:10124000031946298A01CC238A010F248316C7017A
:101250008312831647085C3E840000308000C70A72
:101260000B3047028A158312031D28298316C701F4
:10127000831283164708673E840000308000C70A47
:101280000B3047028A158312031D38298316320852
:10129000C400DB0183128A01B7248316DB018312A9
:1012A0008A013C2483165F085C028A1583120319A5
:1012B0005B298A01142583165D085E028A15831254
:1012C000031964298A01CC2383165D08DE0083128A
:0A12D0008A15F42863008A156A29C4
:02400E00223F4F
:104200004000F3000000C0000700060000000000AE
:104210004D006F006F006E000000530075006E00CF
:1042200020000000200020002000200000004100AD
:104230006E00740065006E006E00610000002000DA
:1042400020005000610072006B0020004F004E0003
:04425000200020002A
:00000001FF
